:1000000000308A00582E0000FF00030E8301A1007B
:100010007F08A0000A08A8008A01A00E0408A20018
:100020007708A3007808A4007908A5007A08A6003C
:100030007B08A700831383128B1E20280B198B29A2
:100040000B1E24288B18B928220884002308F700E7
:100050002408F8002508F9002608FA002708FB0004
:1000600028088A00210E8300FF0E7F0E09000A1067
:100070008A100A11820723342034773469346E34AD
:1000800064346D346F346E343234203400340A10EA
:100090008A100A118207323439342D3444346534DD
:1000A00063342D343034363400340A108A100A1187
:1000B0008207233420346C346F34673420340034A6
:1000C0000A108A100A1182072334203464346C34F5
:1000D0006F34673400340A108A100A1182072334FF
:1000E000203464346C346F346134643400340A1066
:1000F0008A100A118207233420344434693473345B
:10010000703400340A108A100A1182072334203414
:1001100049346E34763461346C3469346434003478
:100120000A108A100A1182072834643429346C3486
:100130006F3467342C342034643428346F342934D9
:1001400077346E346C346F34613464342C3420343E
:1001500064342834693429347334703400340A1018
:100160008A100A11820763346D3464343A342034BF
:1001700000348B12AB0A8B168B108A11242844088A
:10018000003A0319E228013A0319F028033A031947
:10019000FE28013A03190C29073A03191A29013AD2
:1001A00003192829033A03193629013A0319442966
:1001B0000F3A03195229013A03196029033A031926
:1001C0006E297C29831605108312051086130613E9
:1001D00086120612861183168511831285158A29C7
:1001E0008316051083120514861306138616061649
:1001F000861583168511831285158A2983160510A5
:1002000083120510861306178612061286158316AA
:100210008511831285118A29831605108312051012
:100220008613061386120616861583168511831209
:1002300085118A2983160510831205148613061367
:1002400086160616861183168511831285118A2952
:1002500083160510831205108617061386120616DC
:10026000861183168511831285118A29831605103C
:10027000831205108617061386120612861183163E
:100280008511831285118A298316051083120510A2
:100290008613061386160616861583168511831295
:1002A00085158A29831605108312051086130613F7
:1002B00086120612861183168511831285118A29EA
:1002C000831605108312051086130613861606166C
:1002D000861183168511831285118A2983160510CC
:1002E00083120514861706178616061686158316BA
:1002F0008511831285158A2983160510831205142A
:100300008617061786120612861183168511831228
:1003100085158A2900348B12AE0BA1290B122C08EB
:10032000AE002B08AF00AF08031998292D08AF07BE
:100330002F08300203189E292F08B000AB01B1141A
:100340000B16AA1CB029AF08031DA829B403AA29BB
:10035000FF30B400B408031DB029FF30B4006300BF
:100360002A1CE829B11CC229B1102F08C400B2010F
:100370004408093C0318C0290A30C402B20AB8294B
:100380004408B300003031180130003A031DD5296C
:10039000311483160511831205153308C400BF20DC
:1003A0008316851083128510E82931108316851075
:1003B00083128514B208031DE1290A30C400BF204E
:1003C000E4293208C400BF208316051183120511E9
:1003D0008B160B118A11242807309F0083160508FD
:1003E0000330F700F70BF22983121F080C13831652
:1003F0009F01103065000330660083126E2E3E3080
:10040000840000080319132A0130F800F701F70BE4
:10041000072AF80B062A4A30F700F70B0D2A0000CE
:100420000000800B042A0034B6013608372000385B
:1004300003191F2AB60A0C1E1B2A9900152AB60199
:1004400036084720003803192A2AB60A0C1E262A25
:100450009900202A0D300C1E2B2A99000A300C1E00
:100460002F2A99002A08093C031D3F2AA9018B1B4A
:10047000A9178B13C401BF20A91B8B175A2A2A085E
:100480000B3C031D4D2AA9018B1BA9178B130130AF
:10049000C400BF20A91B8B175A2A2A080D3C031D34
:1004A0005A2AA9018B1BA9178B130B30C400BF203C
:1004B000A91B8B1783160511831205110330B60093
:1004C000C830BE00FF21B60B602A831605118312C7
:1004D000051583168510831285100330B600C830C9
:1004E000BE00FF21B60B6F2A831685108312851478
:1004F000872E81010430F700F71D862A073081011D
:10050000813084000008C0390F38800064008130D9
:1005100084000008C039770480008B160B16C030A9
:100520008B04882EC1013F08633C03189B2A64306A
:10053000BF02C10A932AC108031DA12AC0080319DA
:10054000A82A30304107C20042080C1EA52A990093
:10055000C1013F08093C0318B12A0A30BF02C10A91
:10056000A92AC108031DB72AC0080319BE2A3030C2
:100570004107C20042080C1EBB2A990030303F07D9
:10058000C20042080C1EC22A99000034831685104E
:100590008312851483160511831205152A10003461
:1005A0000830F80000000000851383168513000052
:1005B0008312C30D0513031CE02A8316051783124B
:1005C0000318E52A831605138312831685178312F1
:1005D000851BEC2A8316E72AF80BD22A0000851324
:1005E000831685130000051700000000851783128D
:1005F000851BFC2A8316F72AF8010000051B7814D6
:10060000851383168513831205138316051383122E
:1006100000348316051700008517000083120513A8
:100620008316051300008312851383168513A030EB
:100630008312C300D0223E08C100C2013E08C3009D
:10064000D0223D08C300D0223F08C300D022831629
:100650000513000085178312851B302B83162B2B67
:1006600000000000000000008316051700000517B9
:100670000000851700008312051383160513000080
:100680008312851383168513A0308312C300D022F2
:10069000780878184D2B40104E2B4014401C6D2BC1
:1006A000831605170000851700008312851B5A2B3F
:1006B0008316552B0513831605130000831285132B
:1006C00083168513A0308312C300D02278087818CF
:1006D0006B2B40106C2B40144E2B00342A1400342A
:1006E000AA100330BB003B0883169B009C131C140C
:1006F0001A088312BD01BC003C08BD00BC010130DA
:100700003B07BE0083169B009C131C141A0883121F
:10071000BC070318BD0A3C08F8003D08F900790839
:10072000B9007808B800BB013B0855200038031910
:100730009E2BBB0A0C1E9A2B9900942B3908BC00E7
:100740003808BB000130BD003C3084000008BE000A
:10075000BF003D08C00092223B08BF003D08C0001A
:100760009222AA1DC6228316851705178312B70188
:10077000B60137087F3C031C022C3908BC0038083E
:10078000BB00BB08031DC72BBC080319D32B0230C9
:10079000BD00F530BE00FF21BD0BC92B3B0803197E
:1007A000BC03BB03C12B2F08BA000B138B138B1B8D
:1007B000D62B37087F3C031CF12B031DE32B360897
:1007C000FE3C031CF12B01303607BB003708BC0090
:1007D0000318BC0A3C08BE003B08BD00FF30BF0048
:1007E00009233708BE003608BD003A08BF000923B8
:1007F000C0308B042E300C1EFB2B9900B60A031957
:10080000B70AB92B6E2300340B138B138B1B052CEB
:10081000B6013608902000380319132CB60A0C1EB6
:100820000F2C9900092C0D300C1E142C99000A3045
:100830000C1E182C9900B601B608031D372C8C1E0F
:100840001F2C1A08B6000A30BE00FF2136080C1E05
:10085000272C99003608403C0318352C36085A3CA2
:10086000031C352C36082038362C3608B6000D30DF
:100870000C1E382C99000A300C1E3C2C99003608AE
:10088000643C031D512CB701370860200038031960
:100890004E2CB70A0C1E4A2C9900442C0D30AA008D
:1008A0008B2C36086F3C031D632CB70137086B2077
:1008B00000380319602CB70A0C1E5C2C9900562CCA
:1008C0000930AA008B2C3608693C031D752CB70132
:1008D0003708772000380319722CB70A0C1E6E2CCB
:1008E0009900682C0B30AA008B2CB70137088220A6
:1008F00000380319802CB70A0C1E7C2C9900762C2A
:100900000D300C1E812C99000A300C1E852C99008C
:100910000130F800AD2C0D300C1E8C2C99000A30E3
:100920000C1E902C9900023083169B0083122A081B
:1009300083169A001C1583120B08F7008B1383167D
:1009400055309D00AA309D009C149C18A52C1C11AC
:10095000770883128B040030F800F808031D082C78
:100960000230B600FA30BE00FF21B60BB22C8A016D
:100970000028062F0B138B138B1BBB2C2F08B600E4
:10098000C0308B043608BF00C00192220D300C1E0F
:10099000C72C99000A300C1ECB2C9900062F08306A
:1009A000BD007708BE008316051700008517831267
:1009B000851BDC2C8316D72C051B0314051F031085
:1009C000F80D00008316851383128513BD0BD32CFD
:1009D000831605170000831205133E080319F32C34
:1009E0008316051383120000831685178312851B57
:1009F000FB2C8316F62C000085138316851300004C
:100A0000831205138316051383124E2DC622B701D8
:100A1000B60137087F3C031C782D031D132D3608C3
:100A2000FE3C031C782D3708BA003608B90083163F
:100A300005170000851700008312851B212D8316E2
:100A40001C2D0513831605130000831285138316CE
:100A50008513A0308312C300D0223A08BC00BD0128
:100A60003A08C300D0223908C300D02283160517E4
:100A70000000851700008312851B402D83163B2D37
:100A8000051383160513000083128513831685133F
:100A9000A1308312C300D022F701CF2C7808BB000D
:100AA00083160513000085178312851B592D8316A5
:100AB000542D000000000000000083160517000000
:100AC00083123B08F8007808B800380F682D782D9D
:100AD0003808BF00C00192220D300C1E6D2D990008
:100AE0000A300C1E712D9900B60A0319B70A092D98
:100AF0006E23062FB90138080F3C0318832D1030E0
:100B0000B802B90A7B2D3908093C031C8F2D3030FF
:100B10003907BA003A080C1E8B2D9900972D4130E9
:100B20003907F63EBB003B080C1E942D990038088F
:100B3000093C031CA32D30303807BA003A080C1EBC
:100B40009F2D9900AB2D41303807F63EBB003B0886
:100B50000C1EA82D990000342C08B8007A250D3001
:100B60000C1EB02D99000A300C1EB42D990083166E
:100B70009B0183122C0883169A001C1583120B0804
:100B8000F7008B13831655309D00AA309D009C14EE
:100B90009C18C82D1C11770883128B0400342D0873
:100BA000B8007A250D300C1ED32D99000A300C1E8A
:100BB000D72D9900013083169B0083122D088316D0
:100BC0009A001C1583120B08F7008B1383165530FF
:100BD0009D00AA309D009C149C18EC2D1C117708D8
:100BE00083128B0400348C1EF32D1A08B9003908C7
:100BF0000C1EF82D99003908393C031C042E3030A6
:100C00003902F800142E142E3908603C03180F2EF8
:100C100039087A3C031C0F2E3908DF39102E3908A9
:100C2000BF3E0A3EF800142E0034F3257808B800C1
:100C3000F3257808B7003708DD3C031D232E38085C
:100C4000F8002B2E2B2E380EF700F030F705770822
:100C50003707F8002B2E003415267808B6008316C7
:100C60009B009C131C141A088312B700B8007A2545
:100C7000062F15267808B60015267808B70036081E
:100C800083169B008312780883169A001C15831222
:100C90000B08F7008B13831655309D00AA309D007A
:100CA0009C149C18512E1C11770883128B04062F5C
:100CB00084011F30830583168E1519309900263064
:100CC000980090308312980007309F00B201B30162
:100CD000FF30B400AF01B001AB01EC290230831644
:100CE0009B009C131C141A088312AA0083169B01F4
:100CF0009C131C141A088312AC00AE00013083163A
:100D00009B009C131C141A088312AD00142A792A24
:100D10002A1DA12E023083169B0009309A001C1553
:100D200083120B08F7008B13831655309D00AA30F1
:100D30009D009C149C189A2E1C11770883128B041A
:100D40007023B6013608AF2000380319AC2EB60A5E
:100D50000C1EA82E9900A22E8C1EAC2E1A08B500CF
:100D600035080C1EB12E99000D300C1EB52E9900C1
:100D70000A300C1EB92E99003508403C0318C72EC6
:100D800035085A3C031CC72E35082038C82E3508B4
:100D90006D3A0319E72E1E3A0319E82E143A031987
:100DA000E92E173A0319EB2E5D3A0319EC2E063A99
:100DB0000319EF2E703A0319F22E063A0319F52E95
:100DC0002F3A0319F82E053A0319F92EFA2E042C9E
:100DD000BA2C7023062F062DAC03AC25062FAC0AC7
:100DE000AC25062FAD03CF25062FAD0ACF25062F44
:100DF0002C2E392E3F300C1EFB2E99000D300C1E70
:100E0000FF2E99000A300C1E032F9900A12E6300BB
:0A420000CC000200090000003C00A1
:02400E00103F61
:08400000030000000E000300A4
:00000001FF
